:020000040800F2
:10000000A832002085010008153E00088D2A00084E
:10001000113E0008FD020008F9540008000000002D
:10002000000000000000000000000000394200084D
:100030006F10000800000000B53E00086143000892
:100040009F0100089F0100089F0100089F01000810
:100050009F0100089F0100089F0100089F01000800
:100060009F0100089F0100089F0100089F010008F0
:100070009F0100089F0100089F0100089F010008E0
:100080009F0100089F0100089F0100089F010008D0
:100090009F0100089F0100089F0100089F010008C0
:1000A0009F0100089F0100089F0100089F010008B0
:1000B0009F0100089F0100089F0100089F010008A0
:1000C0009F0100089F0100089F0100089F01000890
:1000D0009F0100089F0100089F0100089F01000880
:1000E0009F0100089F0100089F0100080000000018
:1000F0000000000000000000000000000000000000
:1001000000000000000000009F0100089F0100089F
:100110009F0100089F0100089F0100089F0100083F
:100120009F0100089F0100089F0100089F0100082F
:100130009F0100089F0100089F0100089F0100081F
:100140009F010008B9040008E90400089F010008A5
:10015000DFF80CD000F04CF800480047E9560008E2
:10016000A8320020EFF30980704780F309887047B8
:10017000EFF30880704780F30888704740BA7047F3
:10018000C0BA70470648804706480047FEE7FEE7CA
:10019000FEE7FEE7FEE7FEE7FEE7FEE7FEE7FEE737
:1001A000214400085101000840EA01039B0703D0E5
:1001B00009E008C9121F08C0042AFAD203E011F8A6
:1001C000013B00F8013B521EF9D27047D2B201E068
:1001D00000F8012B491EFBD270470022F6E710B54C
:1001E00013460A4604461946FFF7F0FF204610BDA5
:1001F000064C074D06E0E06840F0010394E8070074
:1002000098471034AC42F6D3FFF7A6FF205A0008F7
:10021000405A00080FB470B5049D9DF81A000828D4
:1002200002DD08208DF81A000C49049808609DF83A
:100230001A008872002407E00DF11B00015D0748D9
:100240000B300155601CC4B29DF81A00A042F3DCCB
:10025000284600F005F870BC5DF814FB802A0020E9
:1002600070B5044603254FF6D0702040B0F5806F7E
:1002700004D1012500201149086010E040F2DF7030
:10028000844203D040F20B70844204D10225002046
:100290000A49086003E00325002008490860012D91
:1002A00004D0022D03D0032D05D103E004E002F0B9
:1002B000EBFE01E000E000BF00BF70BDF0000020D9
:1002C00010B501214FF0C05003F0F6FD012003F0FE
:1002D000EBFD10BD00BF0748006800F4E060064970
:1002E0000843001D03490860BFF34F8F00BF00BFE4
:1002F000FEE700000CED00E00000FA0500BFFEE79D
:1003000002480068C043014908607047D8000020D7
:1003100000B50648006838B901200549086005485D
:100320000249086005F0EAF800BD0000E000002086
:10033000DC0000202083B8ED4FF0FF300149086059
:1003400070470000D800002030B503460C4609482D
:100350000268002108E0605C5040C5B2064850F8D1
:10036000250080EA1222491C9942F4D30148026018
:10037000002030BDD80000208026002000B589B0C4
:100380000121092003F0B8FD0121480603F094FD86
:100390000121880603F090FD4FF40050ADF82000D5
:1003A00003208DF8220018208DF8230008A940486A
:1003B00002F08FFA4FF48050ADF8200048208DF8FD
:1003C000230008A93A4802F084FA00208DF81A00A8
:1003D00001208DF81B0000208DF81C008DF81D00F9
:1003E0008DF81E008DF81F008DF8160001208DF885
:1003F000170008208DF8180001208DF8190006203C
:10040000ADF8140005A92B4800F0B9FA0E208DF8BC
:100410000E0000208DF80F0001208DF81000002044
:10042000ADF80400ADF80600ADF80800ADF80A001C
:100430000120ADF80C008DF8110001A800F046F97C
:10044000012210211B4800F091FA41208DF8000094
:1004500001208DF8010000208DF8020001208DF8A8
:100460000300684603F0DEFC012005F0A9F8012234
:100470005102104800F07AFA012291020D4800F072
:1004800075FA0122D1030B4800F070FA42208DF872
:10049000000001208DF8010000208DF802000120ED
:1004A0008DF80300684603F0BDFC002009B000BDD4
:1004B000000C01400068004000B587B0012005F045
:1004C0008BF802AA0121074800F0E3FA0698009091
:1004D00002A80FC8FFF79EFE142102A8FFF77DFEB9
:1004E00007B000BD0068004010B54FF400712D4802
:1004F00000F0ACF9012820D12B492A4800F06AF914
:10050000012815D100BF022808DA284911F8301057
:1005100021B1264911F83010032900D104E002214D
:10052000224A02F8301000BF1F491E4800F042F86E
:100530004FF400711B4800F059F84FF480611948DE
:1005400000F084F901282BD11749891C154800F0C7
:1005500041F901281FD10124022C03DA134810F8B5
:10056000340000B912E00320104901F8340001EB17
:10057000C401081D002103F0A1FF1CB90C4800F0C4
:1005800089F802E0074800F085F800BF0649891C99
:10059000044800F00FF84FF48061024800F026F89C
:1005A00010BD0000006800400200F010FC000020B8
:1005B0000064004000220C4B994202D10023836169
:1005C00011E0C1F3130201F000730BB1C2600AE045
:1005D00001F080630BB1026105E001F000630BB133
:1005E000826000E0426070477000F030B1F5007F3B
:1005F0003AD00FDC202928D006DC01291CD00429A0
:100600001DD0082940D11DE0402921D0B1F5807FBF
:100610003AD126E0B1F5004F31D006DCB1F5806F5C
:1006200025D0B1F5006F2FD124E0B1F5803F12D075
:10063000B1F5003F28D111E0154A826025E008227B
:10064000C26022E01022C2601FE0082202611CE0AA
:100650001022026119E00822426016E01022426076
:1006600013E00422426010E0042242600DE0042204
:1006700042600AE0002282610422426005E000221A
:1006800082610422426000E000BF00BF70470000AA
:100690000101010010B504460B48844209D1012133
:1006A000480603F019FC00214FF0007003F014FC21
:1006B00008E00121880603F00FFC00214FF0806064
:1006C00003F00AFC10BD00000064004010B50021DA
:1006D000837A012202FA03F13D4A126842F00102D4
:1006E0003B4B1A603A4A1C3212688A43384B1C331F
:1006F0001A60027BCAB9364A0C3212688A43344BFC
:100700000C331A604288C38842EA0343304A4032BD
:10071000847A42F834300288838842EA03432C4AC0
:100720004032847A02EBC4025360027B012A19D161
:10073000274A0C3212680A43254B0C331A60428850
:10074000038842EA0343224A4032847A42F8343032
:10075000C288838842EA03431D4A4032847A02EB0E
:10076000C4025360C27A3AB9194A121D12688A4308
:10077000174B1B1D1A6006E0154A121D12680A432A
:10078000134B1B1D1A60028932B9114A14321268C8
:100790008A430F4B14331A600289012A06D10C4A8E
:1007A000143212680A430A4B14331A60427B012A3E
:1007B00006D1074A1C3212680A43054B1C331A60E3
:1007C000034A126822F00102014B1A6010BD0000BA
:1007D0000066004010B50246002001F4700343B1EA
:1007E0009369C1F3130423400BB101202DE00020D5
:1007F0002BE001F0807343B15368C1F3130423402D
:100800000BB1012021E000201FE001F0006343B1A3
:100810009368C1F3130423400BB1012015E00020BD
:1008200013E001F0007343B1D368C1F31304234014
:100830000BB1012009E0002007E01369C1F31304A4
:1008400023400BB1012000E0002010BD70B504462C
:100850000D46002660692840002871D0B5F5807FDC
:100860005CD010DC082D35D006DC012D20D0022D07
:1008700024D0042D72D127E0102D31D0202D35D079
:10088000402D6BD138E0B5F5004F60D009DCB5F5EF
:10089000007F49D0B5F5806F4CD0B5F5006F5DD1C4
:1008A0004FE0B5F5803F2DD0B5F5003F56D12FE094
:1008B000A0682D4900F0D2FB064651E0E068032114
:1008C00000F0CCFB06464BE0E068082100F0C6FBD8
:1008D000064645E0E068102100F0C0FB06463FE018
:1008E0002069032100F0BAFB064639E0206908219F
:1008F00000F0B4FB064633E02069102100F0AEFBA7
:1009000006462DE06068082100F0A8FB064627E0B7
:100910006068102100F0A2FB064621E0A0690121D9
:1009200000F09CFB06461BE0A069022100F096FB4C
:10093000064615E0A069042100F090FB06460FE092
:100940000FE0A069702100F089FB064608E06068AE
:10095000042100F083FB064602E0FFE7002600BF0B
:1009600000E00026304670BD010101001AB1436964
:100970000B43436102E043698B434361704730B5E9
:10098000024600200023146824F002041460146856
:1009900044F00104146000E05B1C546804F001049E
:1009A0001CB94FF6FF74A342F6D1546804F0010459
:1009B0000CB900206CE08C79012C04D1146844F04F
:1009C0008004146003E0146824F080041460CC797F
:1009D000012C04D1146844F04004146003E014684E
:1009E00024F0400414600C7A012C04D1146844F003
:1009F0002004146003E0146824F0200414604C7A8E
:100A0000012C04D1146844F01004146003E014684D
:100A100024F0100414608C7A012C04D1146844F082
:100A20000804146003E0146824F008041460CC7A0D
:100A3000012C04D1146844F00404146003E0146829
:100A400024F0040414608C78A407CD7844EA05648B
:100A50000D7944EA05444D7944EA05540D886D1E2C
:100A60002C43D461146824F001041460002300E0D6
:100A70005B1C546804F001041CB14FF6FF74A342E0
:100A8000F6D1546804F001040CB1002000E001200C
:100A900030BD10B500F5D87303EB01131B6803F0EC
:100AA00004031372137A53B900F5D87303EB0113DF
:100AB0001B6840F2FF7404EA5353136009E000F529
:100AC000D87303EB01131B686FF0604404EAD3038F
:100AD000536000F5D87303EB01131B6803F00203A6
:100AE000537200F5D87303EB01135B6803F00F0337
:100AF000937200F5D87303EB01135B681B0AD37480
:100B000000F5D87303EB01139B68D37200F5D8731B
:100B100003EB01139B681C0A147300F5D87303EBF5
:100B200001139B681C0C547300F5D87303EB01137D
:100B30009B681B0E937300F5D87303EB0113DB68FE
:100B4000D37300F5D87303EB0113DB681C0A14742C
:100B500000F5D87303EB0113DB681C0C547400F52B
:100B6000D87303EB0113DB681B0E937421B9C368C0
:100B700043F02003C36003E0036943F020030361F3
:100B800010BD10B502460020936803F08063B3F1F6
:100B9000806F00D110E0936803F00063B3F1006F41
:100BA00001D1012008E0936803F08053B3F1805F26
:100BB00001D1022000E00420042874D002F5C073A3
:100BC00003EB00131B6803F0010402F5C07303EB91
:100BD00000131C600B7A7BB94B7A0C8843EA4453B0
:100BE00002F5C07404EB00142468234302F5C074BA
:100BF00004EB0014236010E00B7A4C6843EAC40352
:100C00004C7A234302F5C07404EB00142468234398
:100C100002F5C07404EB001423608B7A03F00F0319
:100C20008B7202F5C07303EB00135B6823F00F04B3
:100C300002F5C07303EB00135C6002F5C07303EBB5
:100C400000135B688C7A234302F5C07404EB001434
:100C500063608B7B1C064B7B44EA03440B7B44EABA
:100C60000323CC7A234302F5C07404EB0014A36081
:100C70008B7C1C064B7C44EA03440B7C44EA032334
:100C8000CC7B234302F5C07404EB0014E36002F54F
:100C9000C07303EB00131B6843F0010402F5C0733B
:100CA00003EB00131C6010BD10B50246002321B1F8
:100CB000012907D002290FD109E090681D4C00EAF4
:100CC00004030BE090681C4C00EA040306E0906803
:100CD0001A4C00EA040301E0002300BF00BF184CD7
:100CE000181BA34216D007DC83B16FF08060184454
:100CF00070B1022818D111E0B0F5007F10D0114C6E
:100D0000204448B1B0F5003F0ED10BE002230DE0C6
:100D100000230BE0002309E0002307E0012305E0A6
:100D2000012303E0012301E0002300BF00BFD8B28C
:100D300010BD0000030000040003000800000310C1
:100D4000000100080001FFF70FB430B585B00024A2
:100D5000142208A96846FFF727FA012004F050FC86
:100D600020B9012005B030BC5DF814FB69460E487F
:100D7000FFF707FF0546002401E0601C84B2012054
:100D800004F03EFC40B129460748FFF78DFF18B933
:100D900040F6FF708442F0DB40F6FF70844201DBD6
:100DA0000120DFE70020DDE70068004010B50020EB
:100DB00000F00AF910BD70473048407820F040003C
:100DC0002E4948700846407820F0200048700846B8
:100DD000407820F0100048700846807820F00F001E
:100DE00088700846807820F0F00088700846007807
:100DF00020F0010008700846007820F00800087014
:100E00000846007820F0040008700846007820F0BA
:100E1000020008700846007820F02000087008469C
:100E2000007820F0100008700846007820F080005C
:100E300008700846007820F04000087008464078A6
:100E400020F0010048700846407820F00200487009
:100E50000846407820F00400487000204871C1F82E
:100E6000F000C1F8F400C1F8F800C1F8FC00C1F8C6
:100E7000EC004FF6FF70A1F8E600704770150020F7
:100E80000148007870470000F600002010B50024EB
:100E9000002012490870124908701249087012495E
:100EA000087072B6FFF788FF00240DE000200F499C
:100EB00008550F4908552146012001F041FE204602
:100EC00001F030FE601CC4B2012CEFDB00F09AF898
:100ED00001F0BEFF03F0A8FD62B610BDF7000020D0
:100EE000F6000020F8000020F5000020F9000020A6
:100EF000FA0000200949097842290DD107494978AB
:100F00004F2909D105498978452905D10349C9786F
:100F1000522901D1012000E0002070478E000020FE
:100F200010B506480078002806DD04480078401E09
:100F30000249087003F0D2FC10BD0000F800002048
:100F400002480078401C014908707047F6000020F4
:100F50000149087070470000F500002010B5FFF748
:100F60002AFF02F0E5FC04F045F9FFF7E9FFFFF77F
:100F7000D7FF10BD10B503480078012801D104F057
:100F800029F910BDF700002000204FF4AC7000E0FC
:100F9000401E0028FCD1704710B50446012C00DB30
:100FA00010BD44B98021064801F068FD10210548B4
:100FB00001F064FD00E000BF00BF00BFF0E70000EB
:100FC00000100140000C014010B50446012C00DB6C
:100FD00010BD74B91021094801F04EFD8021084868
:100FE00001F04CFDFFF7D0FF8021054801F044FDE2
:100FF00000E000BF00BF00BFEAE70000000C0140B6
:101000000010014010B50020FFF7C6FF10BD000022
:1010100010B500240F480078012817D1FFF79EFF74
:101020000D480068B0F5FA6F0AD3FFF7BFFE06E07F
:10103000601C84B2B4F5487F01DBFFF74BF9F7E79A
:1010400005480068401C0449086002E0012001498D
:10105000087010BDF7000020F000002002460020BC
:1010600002EA01030BB1012000E000207047704745
:101070000120014908707047C200002070B5044685
:10108000012501F0FDFCA04200D10025284670BDDD
:1010900038B502221021684604F0C8FA0546012D31
:1010A00001D0002038BD002409E01DF8040006A18D
:1010B000095D884201D00020F4E7601CC4B2022C14
:1010C000F3DB0120EEE700004852000010B50548B0
:1010D000807800F00F00012802D1FFF7D9FF10BD82
:1010E0000120FCE77015002000200549897801F0F7
:1010F0000F01012901D1012000E00120704700000B
:101100007015002002460020A2F57143843B73B99C
:101110000B78632B01DD012008E04B783C2B01DDCF
:10112000012003E08B781F2B00DD012000E000BFD1
:1011300000BF704770B5054604F0BCFA72B68B2D3F
:1011400006D10E480068012182680D48904711E0E1
:101150002E2D0FD1002404E0AA200A490855601C56
:10116000C4B2082CF8DB054800680822054943682A
:101170000348984704F0A6FA62B670BD2800002024
:1011800000380208A8000020002004E0AA21034A39
:101190001154411CC8B20828F8DB70478E000020AB
:1011A000012802D0022800D000BF7047012802D0D9
:1011B000022800D000BF70472DE9F0410446207995
:1011C000401CC6B22068477820688578032E03DC6F
:1011D000132003F0BBFF44E037B1032F1BD0802F57
:1011E00003D0832F2ED117E000BF042E05D013208B
:1011F00003F0ACFF03F0B6FC32E00220A081032D27
:1012000001DC012D03DA312003F0A0FF02E02846C3
:10121000FFF7CCFF24E000BF042E05D0132003F01D
:1012200095FF03F09FFC1BE00220A081032D01DC51
:10123000012D03DA312003F089FF02E02846FFF791
:10124000AFFF0DE003F006FA18B1802003F0BCFFF9
:1012500005E0002003F0B8FF122003F077FF00BF85
:1012600000BF03F037FCBDE8F08170B5044620797B
:10127000401CC6B22068457825F08005022E03D1B7
:10128000132003F063FF1FE0012D02D0022D0CD1CB
:1012900000E000BF032E05D0132003F057FF03F03A
:1012A00061FC10E00220A0810DE003F0D3F918B139
:1012B000802003F089FF05E0002003F085FF122065
:1012C00003F044FF00BF00BF03F004FC70BD00004A
:1012D00070B50246002028E00D5C2B02002421E0BE
:1012E000134DB5F8E6505D4005F4004555B1104D7D
:1012F000B5F8E65041F2210686EA45050C4EA6F8FF
:10130000E65009E00A4DB5F8E6504FF6FF7606EADA
:101310004505074EA6F8E6504FF6FF7505EA43036C
:10132000651CECB2082CDBDB401C9042D4D370BDB2
:10133000701500202DE9F04105460E4617464FF086
:1013400000081448807800F00F00012805D01148EB
:10135000807800F00F00022814D104F0ABF972B6C7
:101360000D4800683A46314643682846984780460B
:1013700004F0A8F962B6B8F1000F01D1002402E030
:10138000012400E0012414B90120BDE8F08100200F
:10139000FBE70000701500202800002070B504460F
:1013A0002079401CC5B22068467826F08006022DC0
:1013B00003DC132003F0CAFE2FE0012E02D0032E1F
:1013C0001CD10DE0032D05D0132003F0BFFE03F068
:1013D000C9FB04E00220A0810A20114908701BE02B
:1013E000032D05D0132003F0B1FE03F0BBFB04E096
:1013F0000220A0810A200B4908700DE003F02AF9B1
:1014000018B1802003F0E0FE05E0002003F0DCFED0
:10141000122003F09BFE00BF00BF03F05BFB70BD1A
:1014200044000020450000202DE9F05F06460F46ED
:1014300090461B48B0F8E84000252BE04FF44830B8
:10144000B5FBF0F100FB115010B9404603F02EFA45
:1014500017F805B04FEA0B294FF0000A16E084EAAE
:10146000090000F4004028B141F2210080EA440064
:1014700084B203E04FF6FF7000EA44044FF6FF70B9
:1014800000EA49090AF1010000F0FF0ABAF1080F69
:10149000E5DB6D1CB542D1D32046BDE8F09F0000CE
:1014A00070150020704710B50346002003E01C5C57
:1014B0000C54441CE0B29042F9DB10BD10B5034659
:1014C000002002E00C5C1C54401C9042FAD310BD7A
:1014D0001D48007820F0800080301B4908700020F3
:1014E000C1F8EC00C1F8F400C1F8F00008464078FB
:1014F00020F0010048700846007820F002000870D3
:101500000846007820F0040008700846007820F0B3
:10151000200008700846007820F001000870084696
:10152000007820F0080008700846407820F010008D
:1015300048700846807820F00F0088700846807850
:1015400020F0F000887070477015002070B50646D6
:101550000C461546224629463046FFF7AFFF70BDC0
:101560002DE9F04F9BB007464FF00008C34600241A
:101570003879401C00F0FF0801201A90B8F1040FE0
:101580000FD0B8F1060F0CD0B8F1080F09D0B8F1A0
:101590000A0F06D0B8F10C0F03D0132003F0D6FDCC
:1015A00083E04FF0010BBBF1050F01DD4FF0050BA0
:1015B000012400255BE0012101EB45013868405C16
:1015C0000DF804001DF804004FEA002A601CC4B2A4
:1015D000022101EB45013868405C0DF804001DF85C
:1015E000040040EA0A0A601CC4B2002019900026D8
:1015F0002DE0304800EB06100088504525D1012031
:1016000019902C4800EB0610407A012803D12A4992
:1016100051F8260080474FF000090DE0254800EB07
:101620000610406810F809000DF80400601CC4B2F0
:1016300009F1010000F0FF091E4800EB0610007AD6
:101640004845EBDC00201A9003E0701CC6B2052E62
:10165000CFDB00BF03F050F910B100201A9008E072
:10166000199810B901201A9003E0681CC5B25D45B5
:10167000A1DB00BFBC81012505E01DF80500B968AC
:101680004855681CC5B2A542F7DB1A9801280CD151
:1016900002F0E0FF18B1802003F096FD05E0002085
:1016A00003F092FD312003F051FD03F013FA1BB05B
:1016B000BDE8F08FB8590008085A0008002005E07E
:1016C0000449095C044A1154411CC8B20528F7DBDF
:1016D0007047000033580008B0000020002005E0EB
:1016E0000449095C044A1154411CC8B20928F7DBBB
:1016F000704700002A5800083D150020002004E033
:10170000FF21034A1154411CC8B20628F8DB704778
:10171000B500002070470000002005E00449095C86
:10172000044A1154411CC8B20928F7DB7047000075
:1017300021580008341500202DE9FC410446257984
:1017400020684678206887780B2D03D0132003F09B
:10175000FDFC46E10EB9442F03D0312003F0F6FC26
:101760003FE1C5480078C0F3400018B1702003F095
:10177000EDFC36E12068C0788DF80400206800791F
:101780008DF80500206840798DF806002068807982
:101790008DF807002068C0798DF800002068007A75
:1017A0008DF801002068407A8DF802002068807A68
:1017B0008DF803009DF8040000069DF8051000EB6D
:1017C00001409DF8061000EB01209DF80710084429
:1017D000A949C1F8F8009DF8000000069DF8011025
:1017E00000EB01409DF8021000EB01209DF8031072
:1017F0000844A149C1F8FC0008460078C0F3C000C5
:10180000002857D10846D0F8FC00B0F5805F0AD810
:101810000846D0F8F800401C28B10846D0F8F80077
:101820009649884203D0312003F090FCD9E09248D9
:10183000D0F8F8009149884207D18F48807820F08D
:10184000F00010308C4988700CE08B48D0F8F8001C
:101850008B49884206D18848807820F0F0002030FB
:10186000854988708448007820F008000830824953
:1018700008700846007820F00200801C08700020E4
:10188000C1F8EC00C1F8F000C1F8F4004FF6FF70A9
:10189000A1F8E6002020A16848700420A1688870A3
:1018A0000020A168C8700420A081FEF731FDFEF77A
:1018B00043FD96E07048D0F8F800724988420FD096
:1018C0006D48D0F8F800B0F5601F09D06A48D0F82C
:1018D000F800B0F1805F03D0312003F037FC7AE0EC
:1018E0006548D0F8F8006749884205D16248D0F8C9
:1018F000FC00B0F5CC3F17D85F48D0F8F800B0F541
:10190000601F05D15C48D0F8FC00B0F5002F0BD863
:101910005948D0F8F800B0F1805F09D15648D0F8A6
:10192000FC00B0F1806F03D9312003F00FFC52E0CE
:1019300051484078C0F3800018B9222003F006FC1B
:1019400049E04D48D0F8F8004E49884207D14A484E
:10195000807820F00F00401C474988701AE0464804
:10196000D0F8F800B0F5601F07D14348807820F028
:101970000F00801C404988700CE03F48D0F8F80008
:10198000B0F1805F06D13C48807820F00F00801CC9
:10199000394988703848007820F00200801C3649A8
:1019A00008700020C1F8EC00C1F8F000C1F8F400A4
:1019B0004FF6FF70A1F8E6002020A16848700420CF
:1019C000A16888700020A168C8700420A081FEF77B
:1019D0009FFCFEF7B1FC2848007820F0080026495B
:1019E000087002F089FF98B32348007820F00200C5
:1019F000214908700846007820F040000870084629
:101A0000007820F0800008700846407820F001003F
:101A100048700846807820F00F008870084680786B
:101A200020F0F00088700020C1F8F800C1F8FC0038
:101A3000C1F8F4004FF6FF70A1F8E6000020C1F8ED
:101A4000EC00C1F8F000887500210B48C1750176E3
:101A50000948007820F010000749087008464078CF
:101A600020F0100048700846407820F020004870B0
:101A700003F030F8BDE8FC817015002000F0002074
:101A800000D8BFFE00A000082DE9F04105460E4633
:101A900000270F48854214D1B6F5CC3F11D803F08A
:101AA00009FE72B60B4800683321826808489047E7
:101AB000074603F007FE62B60FB9002402E00124D6
:101AC00000E0012414B90120BDE8F0810020FBE70B
:101AD00000A000082800002070B504464FF6FF76ED
:101AE0002579012D03D0132003F030FB86E0454813
:101AF000007800F0010040B142484078C0F3800017
:101B000018B9222003F022FB78E03E480078C0F3A9
:101B1000400020B13B484078C0F3001018B92420A1
:101B200003F014FB6AE03748007820F01000103012
:101B3000344908700846407820F010004870084684
:101B4000007820F0200008700846007820F002009D
:101B500008700846407820F0040048700846407835
:101B600020F02000487000204871C1F8EC00C1F856
:101B7000FC00C1F8F8000846007800F0010010B938
:101B80000020C1F8F4001F480078C0F3C00018B16D
:101B90001C48B0F8E6602DE01A48807800F00F008D
:101BA000012808D117493722D1F8F4001649FFF768
:101BB0003BFC06461EE01348807800F00F00022828
:101BC00009D110493722D1F8F4004FF46011FFF722
:101BD0002BFC06460EE00B48807800F00F00022830
:101BE00008D108493722D1F8F4004FF08051FFF7AF
:101BF0001BFC0646FEF784FB0120A08102F06AFF71
:101C000070BD00007015002000A000082DE9FC5FE9
:101C100004464FF0000B2579206846782068C0788C
:101C20002168897800EB01201FFA80FA042D06DA7A
:101C3000132003F08BFA02F04DFFBDE8FC9F5046E5
:101C4000BAF57F4F73D009DCA0F2022040B3A0F5B3
:101C50005C40A0F5EF7000286AD107E06FF47F4187
:101C60000844002877D00128F6D168E002F036FE5B
:101C7000032803D07F2003F069FA10E0052D03D07C
:101C8000132003F063FA0AE0012E03D0122003F0C0
:101C90005DFA04E00020A16808710520A08169E1D7
:101CA0002068007900062168497900EB014021682D
:101CB000897900EB01202168C97900EB0109082D21
:101CC00003D0132003F042FA38E0012E03D0122093
:101CD00003F03CFA32E0AA480078C0F3001018B9CB
:101CE000222003F033FA29E0312002F0DFFD4846DC
:101CF000FFF7C4F9E8B9A248807800F00F00012886
:101D000002D19F49C87002E001209D4908719C489A
:101D1000007820F010009A4908700846007820F0FA
:101D20000100401C08700020A168087104E025E053
:101D300012E10120A16808710520A0811AE102F0DA
:101D4000CDFD032808D002F0C9FD022804D07F2071
:101D500003F0FCF911E0B7E0042D03D0132003F0E9
:101D6000F5F90AE0012E03D0122003F0EFF904E0A8
:101D70000020A16808710520A081FBE00D2D03D192
:101D800020680079442803D0132003F0DFF99AE09B
:101D9000012E03D0122003F0D9F994E02068407995
:101DA0008DF80400206880798DF805002068C079DE
:101DB0008DF806002068007A8DF807002068407AC8
:101DC0008DF800002068807A8DF801002068C07AC4
:101DD0008DF802002068007B8DF803009DF8040058
:101DE00000069DF8051000EB01409DF8061000EB81
:101DF00001209DF8071047189DF8000000069DF887
:101E0000011000EB01409DF8021000EB01209DF84D
:101E1000031000EB01085B48874251D1B8F5CC3F75
:101E200005D8574880780121B1EB101F18D05448CD
:101E3000007820F00200524908700846007820F02F
:101E4000080008700846407820F0400048700846B6
:101E5000807820F0F0008870312003F077F932E0CC
:101E6000312002F023FD41463846FFF70DFE0128E0
:101E700022D14348407820F00400001D40494870BA
:101E80000846407820F0400048700846407820F02E
:101E90000800487000F06AFA8B20FFF74BF9002029
:101EA000A16808710520A0813548007820F0010064
:101EB000401C3349087006E0722003F047F902E045
:101EC000312003F043F955E0042D03D0132003F033
:101ED0003DF940E0012E03D0122003F037F93AE03B
:101EE00027484078C0F3801018B9222003F02EF95B
:101EF00031E0FFF7EBF8012821D1FFF7F5F80128D1
:101F00001DD11F480079012819D11D48C07801282A
:101F100015D1FFF739F92E20FFF70CF91848407852
:101F200020F008000830164948700020A1680871A8
:101F30000520A081002012490871C87002E022200B
:101F400003F004F900200E49C1F8F4000846807837
:101F500020F00F0088700DE002F07CFB18B18020AB
:101F600003F032F905E0002003F02EF9312003F0F0
:101F7000EDF800BF00BF02F0ADFD00BF5DE6000060
:101F80007015002000A000082DE9FE43054602F070
:101F9000ABFC07462879401CC6B2286890F801803F
:101FA000022E03DC132003F0D1F8CDE1B8F1010FCC
:101FB00009D0B8F1020F6CD0B8F1050F6FD0B8F1AD
:101FC000060F6DD13EE1012F03D17F2003F0BEF853
:101FD0005EE0032E03D0132003F0B8F858E0DC488D
:101FE000007801280ED1A9684870002405E000217E
:101FF000A01CAA681154601CC4B2042CF7DB062094
:10200000A88145E0D348007A012803D0D148807ADE
:10201000012803D1372003F099F839E00120A9689D
:102020004870CD480078012812D1CA48007B0328A7
:102030000EDB362003F08AF80120C64988720020A2
:102040008880C648007810B90120C44908707AE138
:10205000C148007810B9C24802F0BEF8002406E07A
:10206000BF48015DA01CAA681154601CC4B2042CB6
:10207000F6DB02ABBB4A0421B94802F025F8002088
:10208000B449087208800120B34908700620A8816D
:1020900059E1012F05D17F2003F058F868E068E08E
:1020A00043E1072E03D0132003F050F860E0AA4864
:1020B0000078012859D10020A7490870A548807AE6
:1020C000012803D1362003F041F849E0002406E05E
:1020D000A01C2968085C0DF80400601CC4B2042C24
:1020E000F6DB9DF800008DF804009DF801008DF8E6
:1020F00005009DF802008DF806009DF803008DF89C
:102100000700042201A9974801F0CCFF90B10220FA
:10211000A9684870A881002003F01EF801208C49AE
:10212000087000208D4908708A49087302208E4982
:10213000087015E0352003F009F88648007B401C44
:10214000844908730846007B032809DB0120887254
:10215000002088808148007810B901207F490870EC
:1021600000207C490880087202E0242002F0EEFF83
:10217000E9E0012F03D17F2002F0E8FF61E0032EA8
:1021800003D0132002F0E2FF5BE0714840780128A1
:102190000FD10520A9684870002405E00021A01C8B
:1021A000AA681154601CC4B2042CF7DB0620A88175
:1021B00047E06848407A012803D06648C07A012881
:1021C00003D1372002F0C2FF3BE00520A968487028
:1021D00061484078012812D15E48407B03280EDB1D
:1021E000362002F0B3FF01215A48C1720021C1809C
:1021F0005A48407810B9012058494870A3E0564821
:10220000407810B9564801F0E7FF002406E0544832
:10221000015DA01CAA681154601CC4B2042CF6DB3A
:1022200002AB504A04214E4801F092FF0021494878
:1022300041720020474948800120474948700620E4
:10224000A88180E0012F03D17F2002F07FFF6BE0A7
:10225000072E03D0132002F079FF65E03E48407856
:1022600001285ED100203C4948703A48C07A0128D4
:1022700003D1362002F06AFF4CE0002406E0A01CE7
:102280002968085C0DF80400601CC4B2042CF6DB5D
:102290009DF800008DF804009DF801008DF8050000
:1022A0009DF802008DF806009DF803008DF80700E8
:1022B000042201A92B4801F0F5FEA0B10620A9686F
:1022C00048700220A881002002F046FF012020492A
:1022D000487000202149487000211E4841730420A5
:1022E0002149087016E0352002F030FF1948407B84
:1022F000401CC1B217484173407B03280ADB01210F
:102300001448C1720021C1801448407810B90120DE
:102310001249487000200F49488000210D48417241
:1023200002E0242002F012FF0DE002F093F918B150
:10233000802002F049FF05E0002002F045FF122056
:1023400002F004FF00BF00BF02F0C4FBBDE8FE8343
:10235000C000002070260020BD0000208C0000205E
:10236000C7000020C3000020C20000204220044912
:1023700008704F204870452088705220C870704700
:102380008E0000202DE9F04705460024A246A14614
:10239000A888801E86B228684778FD4890F8058096
:1023A00008F1010000F0FF08012E02DA132002F00C
:1023B000CDFEB6F5806F03DD712002F0C7FEFCE1B3
:1023C000F3480078C0F3800050B9F148D0F8F0002D
:1023D000B0F5406F04D8EE484078C0F3001070B1FB
:1023E000EB48407820F01000E949487008464078F2
:1023F00020F040004870702002F0A8FEDDE1E448C3
:102400000078C0F3801028B9E14800780121B1EBD1
:10241000D01F03D1722002F099FECEE1DC48007893
:10242000C0F3400018B9242002F090FEC5E1D8485E
:102430004078C0F3401028B9012F03D0732002F078
:1024400085FEBAE1781C804502D10220A881B4E162
:10245000B84503D0732002F079FEAEE1CC48007895
:1024600000F0010040B1CA484078C0F3800018B9BC
:10247000222002F06BFEA0E1C548007820F0200089
:102480002030C34908700846407820F020002030F2
:10249000487008464771007800F0010000287CD0A1
:1024A000002415E0A01C2968085CB949D1F8F01097
:1024B000B84A5054B648D0F8F000401CB449C1F8AE
:1024C000F0000846D0F8F400401CC1F8F400641C89
:1024D000B442E7D32868811C3046FDF735FFAC488D
:1024E000D0F8F400AA49D1F8FC10884277D3A84864
:1024F000D0F8F000B0F5006F2DD3A5494FF400627D
:10250000D1F8F800A349FEF715FF40B9FEF7E0FF48
:10251000722002F01BFE02F0DDFABDE8F0879C4855
:10252000D0F8F80000F500609949C1F8F8000846B5
:10253000D0F8F000A0F50060C1F8F000002405E03C
:1025400004F500609349085C0855641C9048D0F875
:10255000F000A042F4D88E48D0F8F000F0B18C48DA
:10256000D0F8F09005E0FF208A4901F8090009F150
:102570000109B9F5006FF6D385494FF40062D1F82F
:10258000F8008449FEF7D6FE40B9FEF7A1FF72209D
:1025900002F0DCFD02F09EFABFE7A5E000207C49D6
:1025A000C1F8F0000846407820F001004870084665
:1025B000007820F0040008700846007820F0200021
:1025C00008700846407820F04000403048700846C7
:1025D000407820F01000103048707EE0FFE76C4833
:1025E000D0F8F000B0F5006F77D36948407820F05C
:1025F0000100401C664948700846007820F004003D
:10260000001D08704FF40062D1F8F8006149FEF730
:1026100091FE38B9FEF75CFF722002F097FD02F0E0
:1026200059FA7AE75A48007820F080005849087033
:102630000846D0F8F80000F50060C1F8F800084638
:10264000D0F8F000A0F50060C1F8F000002405E02B
:1026500004F500604F49085C0855641C4C48D0F8EC
:10266000F000A042F4D84A48D0F8EC00401C484999
:10267000C1F8EC000846807800F00F00012805D171
:102680000846D0F8EC00B0F5607F17D84048807855
:1026900000F00F00022805D13D48D0F8EC00B0F55D
:1026A000607F0BD83A48807800F00F0002280ED1E6
:1026B0003748D0F8EC00B0F5802F08D9FEF708FFB6
:1026C000722002F043FD02F005FA26E705E03048EB
:1026D000007820F040002E4908702D48007820F046
:1026E00004002B49087066E0B6F5805F58DA0024D4
:1026F0000FE0A01C2968085C2549D1F8F010254A94
:1027000050542348D0F8F000401C2149C1F8F00093
:10271000641CB442EDD31E49D1F8F0001D49FEF708
:10272000D7FD2868811C3046FDF70EFE1848D0F80A
:10273000F400194900EB010A154880780121B1EB3A
:10274000101F0BD10AEB06001449884206D210482C
:10275000104AD0F8F0105046FEF7F8FE0C48D0F8BA
:10276000F4000B49D1F8F01008440949C1F8F4000D
:102770000846D0F8F400D1F8FC10884217D304487A
:10278000407820F010001030014948700FE0000040
:10279000701500207016002000F00020FFFF0020C0
:1027A00000200B49C1F8F400312002F0CFFC0020DA
:1027B0000749C1F8F0000220A8810548007820F000
:1027C00010000349087002F085F900BFA5E600007B
:1027D000701500202DE9F047054695F8048028681B
:1027E000407806022868807806432868C71C4FF0A6
:1027F0000109B8F1030F03DC132002F0A7FC5CE031
:10280000002447E02F4800EB04100088B0423FD17D
:102810002C4800EB0410407A072839D1294800EBF6
:102820000410007AC01C404505D0132002F08EFC35
:102830004FF0000930E039463046FEF763FC0128CE
:1028400005D1312002F082FC4FF0000924E0032082
:10285000A8811C4800EB0410027A1A4800EB04100F
:1028600041683846FEF71FFE164800EB041000884A
:102870004FF28411884208D100F028F812484078BD
:1028800020F00200801C104948704FF0000903E05E
:10289000601CC4B2052CB5DB00BFB9F1010F0CD12F
:1028A00001F0D8FE18B1802002F08EFC05E0002077
:1028B00002F08AFC312002F049FC02F00BF9BDE87D
:1028C000F0870000B8590008701500200146FF206D
:1028D00070472DE9F0410246002500260020002324
:1028E0000024002791F803C00CF00F0591F803C0F5
:1028F0000CF0100CBCF1000F03D091F802C04CEAB0
:10290000050591F800C0BCF1000F31D0146800201B
:102910002BE04FF0010C0CFA00F3B1F800C00CEA08
:1029200003069E4220D183004FF00F0C0CFA03F7F0
:10293000BC4305FA03FC4CEA040491F803C0BCF163
:10294000280F06D14FF0010C0CFA00FCC2F814C09D
:102950000AE091F803C0BCF1480F05D14FF0010C1B
:102960000CFA00FCC2F810C0401C0828D1D3146037
:10297000B1F800C0BCF1FF0F34DD546800202EE038
:1029800000F1080C4FF0010808FA0CF3B1F800C090
:102990000CEA03069E4221D183004FF00F0C0CFA83
:1029A00003F7BC4305FA03FC4CEA040491F803C0A6
:1029B000BCF1280F05D100F1080C08FA0CF8C2F898
:1029C000148091F803C0BCF1480F07D100F1080C46
:1029D0004FF0010808FA0CF8C2F81080401C0828D3
:1029E000CED35460BDE8F081F0B50A460023002440
:1029F0000021002500F00046B6F1004F02D11D4E27
:102A0000F16901E01B4E7168C0F3034583B200F425
:102A10004016B6F5401F08D121F07061154E76685A
:102A200026F07066134F7E6012E000F48016B6F553
:102A3000801F06D1032606FA05F4A14341F0706118
:102A400006E0460D360103FA06F6B14341F0706127
:102A500022B1460D360103FA06F6314300F0004676
:102A6000B6F1004F02D1034EF16101E0014E7160F9
:102A7000F0BD0000000001404161704701617047F6
:102A80000148006870470000D800002000BFFEE742
:102A9000704700002DE9F04F95B004468A469046F5
:102AA0001E460025402105A8FDF797FB0020049055
:102AB0000027012003904FF0000B194800EB441051
:102AC00000680490164800EB44104779FF2E00D0B0
:102AD0003746402F00D94027114800EB4410D0F86A
:102AE0001C90002505E019F8050005A94855681C4B
:102AF000C5B2BD42F7D305ABCDE90074514640469F
:102B0000049A00F029F88346BBF1000F02D101209E
:102B1000039001E000200390039815B0BDE8F08F0A
:102B20003858000810B50446012C06DA0020034985
:102B300008552146012000F003F810BDFB000020DD
:102B4000012803D10122034B5A5402E00022014B19
:102B50005A547047F40000202DE9F04F87B0064624
:102B60008B4617469846DDE910954FF0000A012E76
:102B700003DB012007B0BDE8F08F1F48C0F80490C8
:102B800000201D4948721D4800EB4510007908706F
:102B90001A4800EB4510407C08B1012000E00020FD
:102BA00015498872154800EB4510807C08B101205A
:102BB00000E000201049087200208DF810000297F4
:102BC000084600798DF8120000208DF811000024CD
:102BD00006E018F804100DF113000155601CC4B292
:102BE0009DF81200A042F4DC0698009002A80FC8DD
:102BF000FEF7AAF85046BDE7982A0020385800088A
:102C00002DE9F04106460C46154600270848005DB0
:102C100008B1012C02DB0020BDE8F0812B462246E2
:102C200039463046FFF736FF80464046F4E700005D
:102C3000F400002010B54FF400600B49086002F06A
:102C40004BFD4FF480600849091F086002F044FD05
:102C50004FF480600449086002F03EFD4FF40060CC
:102C60000149091F086010BD140C014010B54FF454
:102C700000600949086002F02FFD4FF480600649AA
:102C8000086002F029FD4FF480600349091D0860C7
:102C900002F022FD10BD0000100C014070B5054689
:102CA0000024002618E06006040E4FF480600F49EF
:102CB000086002F011FD0D480838006800F400605B
:102CC00008B1601CC4B24FF480600849091D086057
:102CD00002F002FD701CC6B2082EE4DB15B9FFF746
:102CE000C5FF01E0FFF7A6FF204670BD100C0140B4
:102CF00070B50446002524E004F0800020B14FF4B4
:102D000000601149086004E04FF400600E49091D9D
:102D1000086002F0E1FC4FF480600B49086002F0AB
:102D2000DBFC4FF480600849091D0860072D02D1C3
:102D30004000091F08606006040E02F0CDFC681C0C
:102D4000C5B2082DD8DB70BD100C014010B54FF492
:102D500000600A4908604010086002F0BDFC4FF4B2
:102D600000600649091D086002F0B6FC4FF480605F
:102D70000249091D086002F0AFFC10BD100C0140B3
:102D800010B54FF40060074908604010091F086043
:102D900002F0A2FC4FF400600249091F086002F033
:102DA0009BFC10BD140C014010B54FF400600E499F
:102DB000086002F091FC4FF480600B49086002F05B
:102DC0008BFC09480838006800F4006008B1012451
:102DD00000E000244FF480600349091D086002F000
:102DE0007BFC204610BD0000100C014010B50446CD
:102DF0000548827A00212046FFF702FF012800D112
:102E000010BD0020FCE700001C15002070B5054631
:102E10000C46224600212846FFF7F2FE012800D189
:102E200070BD0020FCE7000010B50446044800789F
:102E300010B900F0E1FD01E000F034FC10BD00002D
:102E40006600002010B500F04DFC00F01DFE10BD26
:102E500010B50020044908710449C870FF200449D6
:102E60000870FFF7EFFF10BD600000205A0000203F
:102E7000660000203EB57948006878498988084492
:102E800001907748C078052806D0062834D0072856
:102E900076D0082875D1A1E07048C088082817DBD3
:102EA00000207049096808706C4880796D4909688C
:102EB00048706C480068801C00906848C088ADF875
:102EC00008006649C988891C88B200F00DFD12E02F
:102ED0006248807963490968087062480068401C4C
:102EE00000905E48C088ADF808005C49C988491C5C
:102EF00088B200F0F9FCA8E05849C88800F0F4FC5A
:102F00005648C088B0F5805F3CDB10205549096801
:102F10000870544800680078524909680870002019
:102F20005049096848704D48C08800164D490968E5
:102F3000887000204B490968C8704848C088000A5A
:102F400048490968087145488079464909684871C7
:102F500044480068801D00904048807A801F80B2FD
:102F6000ADF808003D48807A801F3C4988800846BB
:102F7000408920F4706048810020394988702CE035
:102F80002DE060E010203749096808703548006876
:102F900000783249C988C1F30321084331490968DF
:102FA00008702E4880792F49096848702D480068BC
:102FB000801C00902948807A801E80B2ADF80800FD
:102FC0002648807A801E254988800846408920F45A
:102FD0007060488100202249887036E000BF2020C0
:102FE0002049096808701F48006800781B49498912
:102FF000C1F3032108431B49096808701948006898
:10300000401C00901648C078082808D11348C08892
:1030100012498988401A80B2ADF8080005E00F48CF
:10302000807A401E80B2ADF808000C488188807A12
:10303000401E084409498880BDF80810491C88B220
:1030400000F052FC01E001203EBD00BF06480168CF
:103050006846884704462046F6E700001C15002015
:103060005A0000206C00002084000020002005E0B1
:10307000AA21044A12681154411CC8B20828F7DB7F
:10308000704700006C00002070B5FE48867A082E5C
:1030900001D0002070BDFB48C07A00F0F00038B1CC
:1030A000102804D020287DD030287CD154E200BFE5
:1030B000F548007998B1F4480079012801D1002041
:1030C000E8E7F048C07A022826D1EE48007B3E2887
:1030D00022D1EC48407B80281ED10020DAE7E94865
:1030E000C07A022818D1E748007B3E2814D1E54871
:1030F000407B802810D1E548008828B9E448008842
:1031000010B9E448007938B10020E0490880012076
:10311000E14908700020BDE700F0E4FA0220DA4936
:1031200008710020DD498880D648C07A00F0F000A0
:1031300000287DD010287CD1D2480088C0F30A0036
:1031400040F2DF71884206D10120CF49087100F0BA
:1031500005FB00209EE7D248C078022807D0D0485F
:10316000C078032803D0CE48C078082806D10120B3
:10317000C549087100F0F2FA00208BE7082E7AD1D9
:10318000C048C07A00F00F004FF6FF7101EA00203E
:10319000C249C8800846C088BA49097B0843BF496C
:1031A000C88001E0DEE06AE20846C088072869DDE1
:1031B00000204881B3480D3008600B46D988B14BD8
:1031C0001B88C3F30A00B74B1A689047B3490860DD
:1031D0000846807A00F0030088B102280ED103204F
:1031E000A9490880072008710846808820F480706B
:1031F00000F58070888000F0BBFA42E000BFA7486D
:103200000068C8B39F48407BA449096808709D487E
:10321000807BA249096848709A48C07B9F49096829
:1032200088709848007C9D490968C870954801E0FD
:1032300035E08FE0407C9949096808719148807CAD
:103240009649096848710620944988800846008993
:1032500020F00F00401C088103208B4908800520C6
:1032600008710846808820F4807000F5807088809E
:1032700000F07EFA04E00BE0FFE7002082490871CD
:1032800000BF0AE001208049087100F067FA04E0FD
:1032900001207D49087100F061FA0020FAE67948C2
:1032A0000088C0F30A00804908807648C07A7B49CC
:1032B000C8800846C088401CB04244DC0846C0882C
:1032C00007283ADC0846C08880B3002048816D4852
:1032D0000C3008600B46D9886A4B1B88C3F30A0080
:1032E000704B1A6890476D49086008460068F0B155
:1032F0000846807A00F00300C8B9002407E061485E
:103300000C30005D654909680855601CC4B263480B
:103310008079401EC0B2A042F1DA01205A490871FA
:103320005E4AD088614A1168884711E005E00120B3
:103330005549087100F012FA0AE00120524908715B
:1033400000F00CFA04E001204F49087100F006FA81
:1033500000209FE601204C49087100F0FFF900BFF2
:1033600000BF8DE147480088C0F30A0040F2DF71DA
:10337000884206D101204449087100F0EFF900208D
:1033800088E641480079032803D03F4800790528A2
:1033900076D13D48007905280FD13B488088C0F39D
:1033A000002040B942490878FFF772FB404908788D
:1033B000FFF73AFD01E000206CE638488088C01D28
:1033C0003649C988884237DB3448C0883349898800
:1033D000401A401CB0420EDC2A48C07A00F00F00B0
:1033E0002E49097A01F00F01884205D001202649B3
:1033F000087100F0B3F9ACE000240AE021480C3079
:10340000005D26490968254A928811440855601CC8
:10341000C4B2224881790079401C081AC0B2A04287
:10342000ECDA012018490871002008801B4AD08876
:103430001E4A116888478CE0082E0BD11148C07ACB
:1034400000F00F001549097A01F00F01884202D0FF
:1034500000F048F97DE00B48017B104800680F4AF6
:10346000928881540748407B0C4909680B4A92882E
:10347000114448700348807B08490968074A19E0ED
:1034800069E00000802A0020600000205200002037
:10349000540000204800002056000020281500207D
:1034A0005A0000207C0000205800002070000020FE
:1034B000680000209288114488707348C07B73496B
:1034C0000968724A92881144C8706F48017C6F483D
:1034D00000686E4A9288104401716B48407C6B49C9
:1034E00009686A4A9288114448716748817C674834
:1034F0000068664A92881044817164488088C01DC3
:10350000624988800846007A401C098960F30301FB
:103510005E4801815E488078B0B15D488078401E89
:103520005B4988700846807870B9052008710320CF
:1035300008800846808820F4807000F580708880BC
:1035400000F016F90020A5E50F205149088003205E
:10355000087100209EE593E04B480088C0F30A0004
:103560004C49098888420ED047480088C0F30A00B9
:1035700040F2DF71884206D101204549087100F010
:10358000EDF8002086E54448C078022807D042487C
:10359000C078062803D04048C07807286ED13E483E
:1035A000007900F00100A0B93B48C078062807D098
:1035B0003948C07807280ED13748807801280AD1C9
:1035C00036490878FFF764FA34490878FFF72CFC8D
:1035D00001E000205EE53048C07802284CD1032E7F
:1035E0004ADB2948C07A302804D0312839D0322823
:1035F0003ED13AE028480079C0F38000F8B9264867
:10360000808820F00400001D234988801E48007B2C
:10361000234908721C48457B0A2D02DA01204872B2
:1036200016E005F0800058B1F02D05DDF92D03DC22
:1036300001201B4948720BE00E201949487207E02F
:1036400005F109000A2190FBF1F0401C1449487271
:103650001348007A10498870012008800320C87040
:1036600009E00F200C49088005E000F00DFA02E0A7
:1036700000F00AFA00BF00BF00200BE500E000BF29
:1036800000BF002006E50000802A00202815002049
:1036900060000020580000205A0000206800002030
:1036A0001C1500200D480079052802D007280DD1EF
:1036B00007E00F200949088003200871FF20C87027
:1036C00005E0002005490880087100E0704700BF50
:1036D000FF200349087000BFF8E7000060000020E9
:1036E0006600002010B518480079012809DD164849
:1036F0000079082805D00820134908711349086883
:10370000804700201049088008710846808820F40E
:10371000807088800846808820F4007088800C487B
:10372000008920F00F000A490881002048810948DB
:103730000078802806D108490878FFF7A9F9FF200A
:103740000449087010BD00006000002074000020D3
:1037500028150020660000206800002010B5FFF743
:10376000C1FF10BD014A508170470000281500209C
:1037700070B538488088C0F34020D8B1354DA8884E
:10378000C0F34020002863D02846808820F40070D1
:103790002946888030490878FFF728FB0446002C2A
:1037A00056D12846808820F4007000F50070294624
:1037B00088804DE027488088C0F30020002847D04B
:1037C000244DA888C0F30020002841D02348007869
:1037D000FF283DD18020214908702846808820F4A8
:1037E00080702946888008201D498872002605E0DF
:1037F000AA201C4909688855701CC6B21848807AEE
:10380000B042F5DC13480079072804D1322015496D
:103810000968087003E03020124909680870002028
:1038200010490968487001200E4909688870002015
:103830000849887008490878FFF7D8FA04463CB967
:103840000448808820F4007000F5007001498880E9
:1038500070BD0000600000206800002066000020AD
:103860001C1500206C00002010B51E4800880028A0
:1038700036D01C4C2088002832D020460088401EBC
:10388000214608800846008840BB08460079032886
:1038900006D0052807D0062809D007281CD103E048
:1038A000FFF720FF19E000BFFFF71CFF15E00D48F0
:1038B000C07810B9FFF716FF0DE003200949088012
:1038C000052008710846808820F4807000F580701B
:1038D0008880FFF74DFF00E000BF01E0FFF748FFE1
:1038E00010BD0000600000200C4A12780C4B03EB66
:1038F00042125179884202DB0A4A91720CE0C2B24C
:10390000094B9A5C094B9A5C064B9A721A46927A5A
:10391000082A01DA08229A72704700006800002025
:10392000385800081C150020CC570008BC57000868
:1039300010B5FFF799FF00F067F910BD10B5034609
:1039400009B9012010BD1648C07808B10320F9E775
:103950001448807A082801DD022200E00122114883
:10396000807A801A80B2884203DB05200C4CE0701C
:1039700002E006200A4CE0700320094C2080094830
:1039800003600020074CA0802046C1800448808846
:1039900020F00100401C024CA0800020D2E7000073
:1039A0005A0000201C15002011484089000A401CC4
:1039B0000F49498960F30B210D4841818188807A44
:1039C000401E80B208440A49C988884203DB0820A7
:1039D0000849C87002E007200649C870032005495D
:1039E00008800846808820F00100401C88807047CD
:1039F0001C1500205A00002010B51F48C07805286B
:103A000006D006280ED0072817D008282CD100E0B1
:103A100000BF1A4801680020884700201649088026
:103A2000C87022E00F20144908800220C8700846A0
:103A3000808820F00400888017E00F48807860B10B
:103A40000D488078401E0C4988700846807820B95F
:103A50000F2008800220C87007E00948407A064914
:103A600008800320C87000E010BD00BFFF2005499A
:103A7000087000BFF8E700005A000020780000201E
:103A80001C1500206600002010B501241B48C078DA
:103A900001280EDD1948C07809280AD009201749E5
:103AA000C870174908688047044614B900201349B4
:103AB000C8700020114908800846808820F0010065
:103AC00088800846808820F00200888054B1002059
:103AD000C8700C4908720846408920F4706048811B
:103AE000082088720848007830B908490878FEF73D
:103AF000CFFFFF200449087010BD00005A000020CD
:103B0000800000201C1500206600002068000020B6
:103B100070B539480079C0F34000D0B1364DA8885F
:103B2000C0F34000002866D02846808820F00200BC
:103B30002946888031490878FFF758F90446002C57
:103B400059D12846808820F00200801C29468880B0
:103B500051E02948007900F0010000284BD0264DA3
:103B6000A88800F00100002845D025480078FF28EB
:103B700041D10020224908702846808820F00100A9
:103B800029468880FFF772FAFFF774F906466EB986
:103B90001A490878FFF72AF9044664BB284680884A
:103BA00020F00200801C2946888024E01248C0785A
:103BB000072807D01048C078082803D00E48C078DE
:103BC00006280ED10C48C078062803D100200D49E4
:103BD000888006E00B488188807A401E081A0949CF
:103BE0008880FF20064908700348808820F0010083
:103BF000401C0149888070BD5A00002068000020E8
:103C0000660000201C15002010B51648008820B35F
:103C1000144C208808B320460088401E21460880A6
:103C200008460088D0B90846C078801E072813D2FD
:103C3000DFE800F00407120C0D0E0F00FFF724FF61
:103C40000BE0FFF7B1FEFFF763FF06E000BF00BF28
:103C500000BFFFF719FF00E000BF01E0FFF758FFCA
:103C600010BD00005A00002008B5074840680090C9
:103C700006490098086004490868FCF77CFA034884
:103C80000068804708BD000000A00008E800002090
:103C900008B501211C2000F02FF94FF40070ADF899
:103CA000000010208DF8030003208DF80200694603
:103CB0005348FEF70EFE4FF400715148FEF7DEFE4A
:103CC0000120ADF8000010208DF8030003208DF8CE
:103CD000020069464A48FEF7FCFD01214848FEF70C
:103CE000CDFE40F20240ADF8000010208DF8030038
:103CF00003208DF8020069464148FEF7EAFD0221E3
:103D00003F48FEF7BBFE4FF480613D48FEF7B4FE2E
:103D1000A020ADF8000010208DF8030003208DF8DE
:103D2000020069463748FEF7D4FD20213548FEF7EA
:103D3000A3FE80213348FEF7A1FE44F22720ADF810
:103D4000000010208DF8030003208DF80200694662
:103D50002D48FEF7BEFD4FF400712B48FEF78EFE96
:103D600001212948FEF788FE02212748FEF784FE3C
:103D700004212548FEF780FE4FF480412248FEF7DB
:103D80007BFE20212048FEF777FE4FF48070ADF8CF
:103D9000000048208DF8030069461948FEF799FD98
:103DA0004FF40070ADF8000048208DF8030069461C
:103DB0001448FEF78EFD0121084600F09DF8012110
:103DC0001248FEF711FE1020ADF8000001208DF81A
:103DD000020010208DF8030069460B48FEF779FDBC
:103DE00010210948FEF74AFE4FF40050ADF80000DC
:103DF00004208DF8030069460248FEF76AFD08BDFD
:103E00000008014000100140000C0140000130009A
:103E100000BFFEE7704710B54FF4A06000F03AF81D
:103E200010BD000070B5002100230F22C47804B338
:103E3000154C246804F4E064C4F5E064210AC1F17F
:103E40000403CA40447804FA03F1847814402143FF
:103E500009010E4C0678A155047804F01F050124D1
:103E6000AC4005786D11AD0005F1E025C5F80041C5
:103E700009E0047804F01F050124AC40044D0678E5
:103E8000761145F8264070BD0CED00E000E400E03E
:103E900080E100E002490143024A116070470000DE
:103EA0000000FA050CED00E00149086270470000CF
:103EB00000000E427047000029B1064AD269024351
:103EC000044BDA6104E0034AD2698243014BDA61B0
:103ED000704700000010024029B1064A12690243EF
:103EE000044B1A6104E0034A12698243014B1A61D0
:103EF000704700000010024029B1064A926902434F
:103F0000044B9A6104E0034A92698243014B9A612F
:103F100070470000001002402DE9F041002100220E
:103F2000002500230026002400278C46DFF860814E
:103F3000D8F8048008F00C0121B1042907D0082921
:103F400059D109E0DFF84C81C0F8008058E0DFF873
:103F50004481C0F8008053E0DFF83481D8F8048051
:103F600008F47012DFF82881D8F8048008F480354E
:103F7000920C0D2A01D0921C00E0062235B9DFF820
:103F8000188102FB08F8C0F8008033E0DFF80081F8
:103F9000D8F82C8008F48036DFF8F480D8F82C802C
:103FA00008F00F0808F1010446B9DFF8E880B8FB13
:103FB000F4F808FB02F8C0F800801BE0DFF8D080BE
:103FC000D8F82C80C8F3031808F10107DFF8C08087
:103FD000D8F82C80C8F3032808F1020CDFF8B4806D
:103FE000B8FBF7F808FB0CF8B8FBF4F808FB02F88C
:103FF000C0F8008004E0DFF89C80C0F8008000BFBB
:1040000000BFDFF88C80D8F8048008F0F0010909BF
:10401000DFF8888018F80130D0F8008028FA03F81B
:10402000C0F80480DFF86880D8F8048008F4E06104
:10403000090ADFF8688018F80130D0F8048028FAFF
:1040400003F8C0F80880DFF84880D8F8048008F446
:104050006051C90ADFF8448018F80130D0F80480B4
:1040600028FA03F8C0F80C80DFF82480D8F8048020
:1040700008F44041890BDFF8288018F80130D0F8A7
:104080000C80B8FBF3F8C0F81080BDE8F0810000A8
:104090000010024000127A0000093D0000000020DC
:1040A0001000002070B503460C460120002107E0F7
:1040B000655C5E5CB54201D0002003E04D1CE9B2B6
:1040C0009142F5DB00BF70BD78B50C46057845B967
:1040D000457835B9857825B9C57815B900251D709D
:1040E00078BD002107E0455C184E765C75400DF800
:1040F00001504D1CE9B20429F5DB9DF8015005F093
:10410000F0059DF8006006F00F0645EA06151570EB
:104110009DF801502D072D0E9DF8026045EA1615F9
:1041200055709DF8025005F0F0059DF8036045EAD2
:10413000161595709DF8035005F00F069DF8005078
:1041400066F31F15D5701C7000BFC9E71C5A000824
:1041500078B50C46057845B9457835B9857825B9DF
:10416000C57815B900251D7078BD002107E0455CB4
:10417000184E765C75400DF801504D1CE9B20429CB
:10418000F5DB9DF8005005F00F069DF8015066F331
:104190001F1515709DF801502D099DF8026006F05D
:1041A0000F0645EA061555709DF8035005F0F00519
:1041B0009DF8026045EA161595709DF8035005F0CC
:1041C0000F059DF8006045EA1615D5701C7000BFFC
:1041D000CAE700001C5A00082DE9F0410446FCF72C
:1041E0004FFE0546134800782844C5B2002612E069
:1041F000691C42F2BB02514343F2390202EB410017
:10420000C11700EB11610912A0EB0127FDB204F800
:10421000015B701CC6B2042EEADB06480078401C25
:104220000449087008460078642801D1002008700D
:10423000BDE8F081E4000020704710B500F002F8FE
:1042400010BD00000CB500200190009040480068AF
:1042500040F480303E49086000BF3D48006800F4EB
:10426000003000900198401C0190009820B94FF652
:10427000FF7101988842F0D13548006800F40030A1
:1042800010B10120009001E000200090009801286A
:104290005CD13048006840F010002E4908600846A4
:1042A000006820F0030008600846006840F0020043
:1042B00008602748406826494860084640684860CA
:1042C0000846406840F4806048600846C06A224959
:1042D00008401F49C8620846C06A204908431C4973
:1042E000C8620846006840F08060086000BF184857
:1042F000006800F000600028F9D01548406820F4FC
:104300007C10134948600846406840F4E810486053
:104310000846006840F08070086000BF0C480068E4
:1043200000F000700028F9D00948406820F0030030
:10433000074948600846406840F00200486000BFF6
:104340000348406800F00C000828F9D10CBD0000BB
:10435000001002400020024000F0FEFF140801009F
:104360000F480068401C0E4908600E480068401C59
:104370000C4908600A4800684FF47A71B0FBF1F20A
:1043800001FB1200012804D107480068401C0649BF
:1043900008600648007810B9012004490870704789
:1043A000340000202C0000203800002030000020C5
:1043B00030B5164800684FF47A72B0FBF2F1B1F1F3
:1043C000807F01D301201DE021F07F40401E4FF08F
:1043D000E022506150170F22002807DA13071D0E44
:1043E0000B4B00F00F04241F1D5503E013071C0E98
:1043F000084B1C5400BF00204FF0E02290610720C2
:104400001061002008B100BFFEE730BD140000209D
:1044100018ED00E000E400E010B5FFF725FC10BD4A
:1044200010B51648006840F00100144908600846BD
:10443000406813490840114948600846006811491E
:1044400008400E4908600846006820F48020086093
:104450000846406820F4FE0048600846006820F0E6
:10446000A05008604FF47F0088600020C862FFF70A
:10447000E4FE4FF000600449086010BD00100240E7
:104480000000FFF0FFFFF6FE08ED00E010B50A485F
:104490000078401C084908700846007803280ADBA9
:1044A00000200870002401E0601CC4B2012CFBDB7A
:1044B00072B6FFF7B1FF10BDEC00002002460023EA
:1044C00021B90D4800681060012070470A48036850
:1044D0001068984205D81068181A884209D301203C
:1044E000F3E71068C0F1FF301844884201D301207F
:1044F000EBE70020E9E70000340000204F48007897
:1045000001280AD14E484089401C4D49488101206C
:10451000087000204949087000E070474848408909
:10452000052190FBF1F201FB120030B944484089AB
:1045300018B101204249487000E0EEE74048408948
:104540000A2190FBF1F201FB120028B93C48408996
:1045500010B101203A49887039484089142190FBF4
:10456000F1F201FB120028B93548408910B1012051
:104570003349C87032484089322190FBF1F201FB87
:10458000120028B92E48408910B101202C49087129
:104590002B484089642190FBF1F201FB120028B9FD
:1045A0002748408910B10120254948712448408995
:1045B0004FF4FA7190FBF1F201FB120028B9204888
:1045C000408910B101201E4988711D4840894FF46F
:1045D0007A7190FBF1F201FB120028B9184840896A
:1045E00010B101201649C8711548408940F2DC51CC
:1045F00090FBF1F201FB120028B91148408910B17B
:1046000001200F4908720E4840894FF4FA6190FB6F
:10461000F1F201FB120028B90948408910B10120CC
:10462000074948720648408941F27071884202DBAE
:1046300000200349488100BF6FE7000030000020E0
:104640000C01002000200249087048804860704733
:104650003C00002003484078022801D10120704727
:104660000020FCE75801002010B504462046FCF766
:10467000A3FD10BD70B53848007900F04000B8B116
:104680003548007920F0400033490871012408467C
:10469000407900B104243148007818B124F00104B5
:1046A00044F0020404F0010010B1002000F05AFDB3
:1046B0002948007902281AD104202749087128487E
:1046C00080680078274948700020244908702448F1
:1046D0008089C82802DA2248858900E0C825EAB224
:1046E0001F4B19699868FCF7DEFE00F049FA1A487A
:1046F000007900F0100068B300201B4908801748BB
:10470000007878280AD11948007838B11348007821
:10471000782814D115484088012810D120200E494E
:1047200008710E48007808B9012000E002200C4909
:1047300088700F490A480161083000F0ADFE074853
:104740000078782806D109480078012802D1022093
:104750000149087170BD0000480000205000002091
:104760005801002070010020520000203C00002071
:104770003D0B002010B504462046FCF776FD10BD29
:1047800070B5044601252289D4E9000100F003F840
:104790000025284670BD03E0531E9AB28B5C8354FB
:1047A000002AF9D1704700002DE9F041044638484D
:1047B000007800F07F072068457825F0800594F8A0
:1047C0000480B8F1010F03D1132000F0BFFC5BE0BF
:1047D000012D04D0022D04D0032D44D100E000BFF0
:1047E00000BFB8F1020F05D0132000F0AFFC00F0BD
:1047F000B9F948E0012F01D1022D03D0022F07D1D2
:10480000032D05D17E2000F0A1FC00F0ABF93AE0C9
:10481000032F04D1022D02D101201D49087100206F
:1048200000F0A0FC002606E000201A4988551A492D
:104830008855701CC6B2022EF6DBFCF719FC062068
:10484000A0810020A16888703220A168C870012072
:10485000A1680871F420A1684871032D02D10120DC
:10486000FCF776FB0FE0FFF7F5FE20B180200B4947
:104870000968C87006E0002008490968C87012205D
:1048800000F064FC00BF00BF00F024F9BDE8F08137
:1048900058010020BD000020C0000020480000207A
:1048A00010B504462046FCF779FD10BD10B504464E
:1048B0000320094908707F204870084684707820DA
:1048C000C870AA20087148718871C8710821002039
:1048D000FEF79CFA10BD0000180100200148007886
:1048E00070470000580100200248007800F07F0067
:1048F0007047000058010020014800787047000010
:10490000500000200A4A127902F0FE02084B1A7188
:1049100049B91A461268824205D11A46127942F004
:1049200002021A7170470122024B1A7000BFF9E7A8
:10493000480000205600002070B504460D46A078BF
:10494000012804D0022803D0032806D104E000BFC8
:10495000284600F057F801E000E000BF00BF00204B
:10496000A07070BD01460120044A127942F0010294
:10497000024B1A711A46116000207047480000204F
:104980002DE9F04104460D46002740F6C41085424B
:1049900003DD0220FEF7E6FE16E040F2DF708442FF
:1049A00003D102200A49487006E040F20B708442AD
:1049B00002D101200649487005488581FFF7D2FFE2
:1049C00006460EB9024887683846BDE8F081000007
:1049D0005801002010B5044600210448FFF792FF5B
:1049E000FEF7BCFE05200249088010BD58010020DA
:1049F0005200002010B503210148FFF783FF10BDCE
:104A0000580100200021054A1180054948714021C4
:104A1000034A11710121034A1170704752000020AE
:104A2000480000205600002010B500201E49887064
:104A300001200870087148710020C8701B48886008
:104A40001B491948016100201A49487108717F20EB
:104A50001949087078208870002018490870184992
:104A60000870FFF7EFFD1748007820F02000154987
:104A7000087000240EE0002113480155801E0155E6
:104A8000001F20F8141000200F490A3921F81400E3
:104A9000601CC4B2022CEEDBFCF7EAFA00200B49E2
:104AA00008800B49088010BD5801002079010020C2
:104AB0003D0B002048000020700100205000002025
:104AC00056000020BB0000207A2600205400002061
:104AD0005200002010B517480079042822D116484A
:104AE0000269846823781548007848B17F201070E7
:104AF000537012480078907003210F48818208E0BB
:104B00000C480068C078802803D003F14000107082
:104B1000521C0A480078782801D0FFF793FD08203E
:104B2000044908710348007940F0100001490871F8
:104B300010BD000048000020580100205000002057
:104B400010B504462046FCF70BFD10BD10B5044619
:104B50002046FCF7F1FD10BD10B504462046FCF7D9
:104B6000BBFF10BD002002490968C87070470000F3
:104B70004800002010B504462046FDF747F810BD58
:104B80002DE9F05F4FF00008F8488468067B207834
:104B9000F749085C00EB4000F64901EB80004578DE
:104BA0002078F349085C00EB4000F24901EB8000FB
:104BB00090F804902078EE49085C00EB4000ED4945
:104BC00001EB800090F805A0FFF78EFE074694F8F1
:104BD00000B02078862800DBC346E7480078C0F3A1
:104BE000401058B1E1484078022807D18020E349BD
:104BF0000968C870FFF76EFFBDE8F09FDC4810F849
:104C00000B00FF2874D0012F04D0022F71D0032F86
:104C100070D14DE0D5484078022848D12078272827
:104C20000ED020782E280BD020782F2808D020787E
:104C3000312805D02078342802D02078372809D1AF
:104C40007F20CF4908708020CC490968C870FFF7E1
:104C500041FFD1E7607800F0800040B32078C4497C
:104C6000085C00EB4000C34901EB8000C078F0B164
:104C70002078192802D02078282804D18020BF4924
:104C80000968C87013E02078B949085C00EB40005F
:104C9000B84911F82000B04205D01320B849087077
:104CA000FFF718FFA8E78020B4490968C8709FE0A3
:104CB000AE48407802284BD1207827280ED02078A3
:104CC0002E280BD020782F2808D02078312805D026
:104CD0002078342802D0207837280CD17F20A849AA
:104CE00008708020A5490968C870FFF7F3FE83E7C4
:104CF000C8E12EE07BE0607800F0800040B32078CF
:104D00009B49085C00EB40009A4901EB8000C078A9
:104D1000F0B12078192802D02078282804D18020EA
:104D200096490968C87013E020789149085C00EB47
:104D30004000904911F82000B04205D0132090495E
:104D40000870FFF7C7FE57E780208C490968C870D4
:104D50004EE086484078022848D1207827280ED097
:104D600020782E280BD020782F2808D020783128C2
:104D700005D02078342802D02078372809D17F2028
:104D80007F49087080207D490968C870FFF7A2FE3E
:104D900032E7607800F0800040B320787449085C06
:104DA00000EB4000734901EB8000C078F0B120783F
:104DB000192802D02078282804D180206F4909685A
:104DC000C87013E020786A49085C00EB400069492C
:104DD00011F82000B04205D0132069490870FFF790
:104DE00079FE09E7802065490968C87000E000BFC6
:104DF00000BF20785E49085C00EB40005D4901EB94
:104E00008000C078002875D0607800F0800000280D
:104E100071D0012E6FDD207828285AD004DC1028AC
:104E200007D0112868D105E03E287CD08528F9D12B
:104E3000D4E000BF607881280ED0607883280BD042
:104E40006078822802D12078112805D060788228E5
:104E50002DD1207810282AD1022E03D013204849C2
:104E6000087035E0FFF740FD012816D1062D01D06E
:104E7000042D09D1002042490870607800F08000BC
:104E80003E490968C87023E0B8F1000F20D14FF007
:104E900001087E203A4908701AE00020384908705D
:104EA000607800F0800035490968C87010E02F482C
:104EB0004078022806D1802030490968C870FFF781
:104EC00009FE99E6607800F080002C490968C870F6
:104ED000CDE0032E11D02548407802280DD123487B
:104EE0004078022841D1802024490968C870FFF722
:104EF000F1FD81E6C1E0BBE0B2E06078802802D03D
:104F00006078832823D1FFF7EFFC012815D1052D08
:104F10000AD100201A490870607800F08000174913
:104F20000968C87021E02DE0B8F1000F1DD14FF0E5
:104F300001087E201249087017E00020104908700F
:104F4000607800F080000D490968C8700DE00748DE
:104F50004078022806D1802008490968C870FFF708
:104F6000B9FD49E612200649087080E0580100208A
:104F7000305900089458000870150020480000209F
:104F8000500000206078802819D1FFF7ADFC01287F
:104F90000BD1042D21D1002060490870607800F009
:104FA00080005F490968C87017E000205B490870FD
:104FB000607800F080005A490968C8700DE05948CF
:104FC0004078022806D1802055490968C870FFF74B
:104FD00081FD11E612205149087048E0022E07D0E9
:104FE00050484078022803D113204C49087036E01D
:104FF0006078812802D06078822822D1FFF774FC83
:10500000012814D1032D09D100204449087060788B
:1050100000F0800042490968C87020E0B8F1000F34
:105020001DD14FF001087E203C49087017E0002098
:105030003A490870607800F0800039490968C87002
:105040000DE038484078022806D1802034490968AC
:10505000C870FFF73FFDCFE512203049087006E029
:10506000607800F080002E490968C87000BF17E022
:1050700000202B490968C87012E0002028490968FF
:10508000C8700DE011202549087026484078022894
:1050900006D1802022490968C870FFF71BFDABE5E7
:1050A0001E48007888BB022D01D1022F07D1032DA5
:1050B00001D1032F03D1052D07D1012F05D17F2069
:1050C00016490870FFF706FD26E01648007900EA49
:1050D000090020B91348407900EA0A0028B13320BA
:1050E0000E490870FFF7F6FC16E005200E4908800F
:1050F00020780E4A105C00EB40000D4A02EB800065
:10510000816808480830884706E0FFE70020044926
:105110000968C870FFF7DEFC00BF6DE55000002095
:10512000480000205801002052000020305900089B
:105130009458000810B504462046FCF725FF10BD22
:10514000014948717047000058010020014908706A
:1051500070470000500000200149087170470000AE
:105160005801002070B5044612488068057811483F
:105170008068407800F07F06012C03D1012000F008
:1051800047F904E0102D02D1304600F041F9FFF755
:10519000ABFB01280CD10020FBF7DAFEFBF778FF10
:1051A000012805D1FBF7A6FE10B90A2002490870B4
:1051B00070BD000058010020440000200149087122
:1051C000704700005801002001490968C870704705
:1051D0004800002010B50348007908B1FFF74AFAEB
:1051E00010BD00004800002010B5FBF711FFFFF7CD
:1051F0004DF910BD10B500F02BF810BD70B5044688
:105200002068457825F080052679012E03D11320EA
:10521000FFF79CFF19E06DB9022E05D01320FFF7B0
:1052200095FFFFF79FFC10E00020A1684870022066
:10523000A0810AE01220FFF789FFFFF793FCFFF738
:1052400009FA10B18020FFF7BFFFFFF743FC70BDE4
:1052500010B56548008818B364480078012806D165
:105260000020624908704FF4FA705F490880604876
:105270000079A8B95C480088401E5B490880084650
:10528000008868B9002008800120FFF76BFF002428
:1052900004E0002057490855601CC4B2022CF8DB1A
:1052A0005348007900F00C00C0B153480088A8B101
:1052B00051480088401E504908800846008868B957
:1052C0004B480068807830B90320494909688870E4
:1052D00000F0CEF802E0012047490880002455E0A4
:1052E000464830F81400B0F57A7F06DB4348001DCD
:1052F00030F81400B0F57A7F46DA4048001D30F8E7
:105300001400401C81B23D48001D20F81410001FFD
:1053100030F81400401C394921F8140001F108004C
:10532000005D012810D1084630F81400B0F57A7FEE
:105330002ADB002021F814000021304808300155F4
:1053400000202F4908551FE02C480A30005D012835
:105350001AD12A48001D30F81400B0F57A7F13DB0B
:105360000020274908550021244808300155001F16
:1053700020F81410801D0155801C005D032803DBFC
:1053800002211E480C300155601CC4B2022CA7DB60
:105390001C480078002809DD1A480078401E194989
:1053A00008700846007808B9FAF794FF16480078A4
:1053B000002809DD14480078401E1349087008468B
:1053C000007808B9FAF786FF10480078002809DD50
:1053D0000E480078401E0D4908700846007808B94C
:1053E000FAF778FF10BD000054000020560000209E
:1053F00048000020C000002052000020702600203D
:10540000BD00002044000020450000204600002090
:1054100010B50446FFF768FA01280AD1FFF7CEFE5F
:1054200004F07F00012810D04FF4FA700B49088077
:105430000BE004F07F00012807D1FFF7BFFE012039
:10544000FFF77EFE0020054908800548047004F03F
:105450007F00012801D1FBF7AFFC10BD54000020F4
:105460005801002010B504462046FCF78BFF10BD04
:1054700010B506490648016103218182083000F019
:105480000BF84FF4FA700349088010BD700100203A
:10549000580100205200002070B5044608480068FA
:1054A000C078802805D0A189A068FEF747FA054694
:1054B00002E00025FFF756FB284600F003F870BD18
:1054C0004800002070B504460CB1032000E0002025
:1054D000054629460148FFF72FFA70BD5801002004
:1054E00010B50320FFF7EEFF002010BD10B50446F5
:1054F0002046FDF76FF910BD00BFFEE7002114E064
:10550000084608220BE00B4B1B68034023B10A4BF3
:105510001B6883EA500000E04008531EDAB2002AFC
:10552000F1DC064B43F82100491C054B1B689942EE
:10553000E6D37047DC000020E00000208026002039
:10554000D000002002E008C8121F08C1002AFAD1CA
:1055500070477047002001E001C1121F002AFBD1F3
:105560007047000008B501210820FEF7C5FC0320A4
:105570008DF8020014208DF803004FF48060ADF820
:10558000000069460D48FDF7A4F903208DF80200DC
:105590004FF40060ADF8000014208DF80300694658
:1055A0000648FDF796F94FF480610448FDF766FA66
:1055B0004FF400610148FDF761FA08BD000C01409D
:1055C000022800DB70470121024A02F8301000BFB8
:1055D000F8E70000FC000020022803DA074911F870
:1055E000301001B970470121044A02F8301000213F
:1055F00002EBC002517000BFF4E70000FC00002085
:105600000146022908DA064810F8310020B10448A2
:1056100010F83100032801D1002070470120FCE779
:10562000FC00002010B5FFF79DFF10BD2DE9F041F3
:1056300007460C461646FDF789FBA020FDF758FBF0
:10564000FDF7B2FB00B130E0A046E11704EB1161B9
:10565000C1F30720FDF74CFBFDF7A6FB00B124E0EA
:10566000E0B2FDF745FBFDF79FFB00B11DE0FDF744
:105670006DFBA120FDF73CFBFDF796FB00B114E0AC
:1056800000250BE0711EA94201D0012100E000219C
:105690000846FDF703FB7855681C85B2B542F1DB7F
:1056A000FDF76EFB0120BDE8F081FDF769FB0020EE
:1056B000F9E70000014802490860704700F0002047
:1056C0002800002003480068006810B1002001494C
:1056D0000860704728000020002001E0411C88B2CB
:1056E0003C28FBDB7047000086B0FEF799FEFAF716
:1056F000E7FDFEF75DFE01A8FEF70EFCFEF78BFB53
:10570000FEF7C6FAFFF78EFFFBF7C0FBFAF736FE8F
:105710004FF400712548FDF7AFF9FBF7B7FBFBF736
:10572000C1FE41E0FEF7EAFE21480078012805D1DC
:1057300000201F49087000F03DF835E01C48407813
:10574000012803D100201A4948702DE018488078BC
:10575000012805D1002016498870FFF745FD23E098
:105760001348C078012803D100201149C8701BE0FC
:105770000F480079012803D100200D49087113E07A
:105780000B484079012803D10020094948710BE0FA
:105790000748C079012807D100200549C8714FF496
:1057A00000710248FDF768F9BCE70000000C0140F9
:1057B0000C01002010B5FBF7DDFB10BD000102035A
:1057C00004050607080C10141820304000010203DD
:1057D0000405060708090909090A0A0A0A0B0B0B3E
:1057E0000B0C0C0C0C0D0D0D0D0D0D0D0D0E0E0EEC
:1057F0000E0E0E0E0E0E0E0E0E0E0E0E0E0F0F0FC6
:105800000F0F0F0F0F0F0F0F0F0F0F0F0F39323139
:10581000343830312D4446303200000000000000A2
:105820000056480012566E00000056480012566E90
:1058300000000001170B10001B0700000008040007
:105840000000020000000000000000000000000056
:10585000292E0008180100200B070000FF07000098
:1058600000000800DF070000FF070000000008003C
:105870002D010000FF0700000000080000000000EC
:105880000000000000000000000000000000000018
:10589000000000000206031000000000A9470008F5
:1058A0000206031000000000A148000803060300E0
:1058B00000000000414B0008060501000000000048
:1058C000355100080303031000000000694600087A
:1058D0001402010001000000ED540008060501005B
:1058E00000000000754B00080B02010001000000E1
:1058F0004D4B0008FF020100010000006554000844
:105900000102010001000000594B000802060310CB
:1059100000000000FD510008020303100000000019
:1059200075470008000000000000000000000000B3
:10593000FFFFFFFFFFFFFFFFFFFFFFFFFFFFFFFF77
:105940000001FFFFFFFFFFFFFFFFFFFFFFFFFFFF64
:10595000FFFF02FFFFFFFF0304FFFFFFFFFF05FF45
:10596000FF06FFFF07FF0809FFFFFFFFFFFF0AFF1A
:10597000FFFFFFFFFFFFFFFFFFFFFFFFFFFFFFFF37
:10598000FFFFFFFFFFFFFFFFFFFFFFFFFFFFFFFF27
:10599000FFFFFFFFFFFFFFFFFFFFFFFFFFFFFFFF17
:1059A000FFFFFFFFFFFFFFFFFFFFFFFFFFFFFFFF07
:1059B000FFFFFFFFFF0B000094F100003D150020EA
:1059C00009010000FFFF000095F10000B500002074
:1059D00006010000FFFF000093F10000B00000206E
:1059E00005010000FFFF00008CF1000046150020BB
:1059F00013010000FFFF000080F1000034150020BB
:105A000009010000FFFF0000DD160008FD16000878
:105A1000BD16000815170008191700083E53E17B52
:105A2000405A000800000020FC0000004455000817
:105A30003C5B0008FC000020AC310000545500081D
:105A40000000000001020304010203040607080924
:105A50000204060800A24A04000000000000000042
:105A6000010203040607080900000000000000000E
:105A70000000000000000000000000000000000026
:105A80000000000000000000000000000000000016
:105A90000000000000000000000000000000000006
:105AA00000000000000000000000000018010020BD
:105AB000D5490008F5490008C55400088149000887
:105AC000E1540008814700080000000000000000C9
:105AD00000000000000000000000000000000000C6
:105AE00000000000000000000000000000000000B6
:105AF00000000000000000000000000000000000A6
:105B00000000000000000000000000000000000095
:105B1000000100000800000000000000000000007C
:105B20000000000000000000000000000000000075
:0C5B300000000000000000000000000069
:04000005080001519D
:00000001FF
